:020000040000FA
:040000001DEF00F000
:0200080014D012
:08001800D8CF81F0E8CF80F0A1
:10002000E0CF82F082C0E0FF80C0E8FF81C0D8FF4F
:100030001000F2B449ED00F011000F01386B396B7C
:100040003A6B3B6B3C6B000E926EC10E936EF00EE2
:10005000946E7C0E956E966A620ED36E800ED56E8F
:1000600000EE00F011EC03F0F28AF28CF28E896A55
:100070008A6A8B6A8C6A8D6A0A0E036E8A8283A4EE
:100080008A8483B48A9483B48A8683A48A963FEF51
:1000900000F0F294032E12000A0E036E83A453EFB5
:1000A00000F08A728C7E83B65DEF00F082BC87EF31
:1000B00000F082BEB1EF00F012008AB873EF00F0DA
:1000C0008ABA77EF00F089B07BEF00F089B27FEF5A
:1000D00000F089B483EF00F089B66FEF00F08996E5
:1000E0008A8856EF00F08A988A8A56EF00F08A9A3A
:1000F000898056EF00F08990898256EF00F089924E
:10010000898456EF00F08994898656EF00F089B80B
:100110009DEF00F089BAA1EF00F08DB0A5EF00F0DF
:100120008DB2A9EF00F08DB4ADEF00F089BC99EF6E
:1001300000F0899C898859EF00F08998898A59EFE5
:1001400000F0899A8D8059EF00F08D908D8259EFE3
:1001500000F08D928D8459EF00F08D94898C59EFC9
:1001600000F08BB0C6EF00F08BB2C9EF00F08BB49B
:10017000CCEF00F08BB6CFEF00F08CB0D2EF00F0F8
:100180008CB2C3EF00F08C928B8012008B908B822C
:1001900012008B928B8412008B948B8612008B96AC
:1001A0008C8012008C908C8212001200000EF86E6F
:1001B000080EF76E050EF66E0800F5503FEF00F0E2
:10060000060E026E130E016EAD0E006E0400002E7B
:1006100006EF03F0012E06EF03F0022E06EF03F0C3
:10062000000CEE6AEAA411EF03F01200280E006E2F
:10063000550E016E040000000000000000000000E4
:100640000000012E1AEF03F0002E18EF03F0120045
:10080000C0F9A4B0999282F88090407924301912EE
:0808100002780010BFA2A3AFA3
:020000040030CA
:0300010028183C80
:02000500BD81BB
:060008000FC00FE00F40E5
:0200000400F00A
:04000000FFFFFF00FF
:00000001FF
